:1000000012C019C018C017C016C01BC015C017C039
:1000100012C011C010C00FC00EC00DC00CC00BC06C
:100020000AC009C008C011241FBECFE5D4E0DEBF5E
:10003000CDBFDCD0BAC2E4CF32BA25BA189528BAFF
:100040001895409A32BA25BA28BA48BE18958895AC
:10005000409BFDCF409808951F93CF93DF93EC0111
:100060009B0119854F81E12FF0E0EE9FC001EF9FCA
:10007000900DFE9F900D11248E0F9F1F642F70E036
:1000800068D2769567952617370728F4411798F4B4
:10009000141B198710C05E81151768F4852F90E036
:1000A0008E1B9F0B242F30E08217930714F459877F
:1000B00002C0410F4987DF91CF911F9108950F939F
:1000C0001F93CF93DF93EC01888581FF2DC00C81B6
:1000D0001D8180FF12C088819981B801681B790B4E
:1000E000CE01BADF8985B801681B71092881398181
:1000F0002617370788F0188613C06A817B81601B3A
:10010000710BCE01A9DF8985B801680F711D2A81A5
:100110003B816217730710F49B0104C081E088875C
:10012000198641983D832C83DF91CF911F910F91C8
:100130000895FC019085892F91FF05C01186809557
:100140008170808702C09260908741980895FC0179
:10015000808581FF12C0759567958681680F711D36
:100160006F3F710519F014F06FEF70E068307105A2
:1001700014F468E070E06683089594E0660F771FDA
:100180009A95E1F72081318180FF14C082819381AB
:10019000860F971F2817390710F0C90101962CE91F
:1001A0008F33920710F08EE39CE9938382839583CB
:1001B00084830895620F731F8FE16034780710F411
:1001C00060E47FE1828193816817790718F0BC01B0
:1001D0006150704071836083758364830895FC016E
:1001E0002481358136952795C90108955F928F92B4
:1001F0009F92AF92BF92CF92DF92EF92FF920F93B6
:100200001F93CF93DF9380E885BF8FEF87BB8EE38B
:1002100084BB80EC81BB9FE3392E8FE382BB86E0F9
:10022000482E222489E18EBD8FE19EE497BD86BDD4
:1002300088E389BF479A80E487B980E690E060E070
:1002400070E048E950E099D18091F7008F3F11F0BC
:1002500081BF03C081B78093F700CC244FE1439561
:1002600001B212B290010426142612BA01BAD49E29
:10027000D12CC49E1D0C60014A9500B232BB21BB3B
:1002800000940422C028469551F71124789401EC7B
:10029000502E88248A94982C11E0A12EB12C01C0F4
:1002A0006701D5DEC09AAD9A8091BE009091BF00E3
:1002B0009695879599BD88BD809164009091650061
:1002C000969587959BBD8ABD80E690E0F8DE80EB31
:1002D00090E0F5DEBCDEC19AAC9A8091D20090919C
:1002E000D3009695879599BD88BD80916E009091B9
:1002F0006F00969587959BBD8ABD8AE690E0DFDE0C
:100300008AEB90E0DCDEA3DEC29AAB9A8091C80053
:100310009091C9009695879599BD88BD8091780088
:1003200090917900969587959BBD8ABD84E790E072
:10033000C6DE84EC90E0C3DE8ADEC39AAA9A80917E
:10034000F0009091F1009695879599BD88BD8091B8
:10035000820090918300969587959BBD8ABD8EE71C
:1003600090E0ADDE8EEC90E0AADE71DEC49AA99A30
:100370008091F0009091F1009695879599BD88BD88
:1003800080918C0090918D00969587959BBD8ABD3C
:1003900088E890E094DE88ED90E091DE58DEC59A22
:1003A000969A8091E6009091E7009695879599BD81
:1003B00088BD8091AA009091AB00969587959BBDD2
:1003C0008ABD82E990E07BDE82EE90E078DE3FDE5F
:1003D000C69A979A8091DC009091DD00969587955A
:1003E00099BD88BD8091B4009091B5009695879590
:1003F0009BBD8ABD8CE990E062DE8CEE90E05FDE12
:1004000056B825DEC79A8091C8009091C90096958C
:10041000879599BD88BD9BBC8ABC86EA90E04FDE7B
:10042000E0E6F0E0808581FD1EC03A9620E0E63FE0
:10043000F207C0F3E19917C0C0E6D0E000E010E099
:10044000C801ABD09881891731F09DBBF894E29A2E
:100450007894E19A08C080E0C73FD80721F0219640
:100460000F5F1F4FEDCF24B135B116B8419B26C0A9
:10047000B9016619770939018091F6008F3040F48F
:100480002AE0829FC0011124805A9F4F60DE1DC068
:1004900075956795759567958091F700680F711D43
:1004A0006F3F710519F014F06FEF70E077FF02C035
:1004B00060E070E06093F70061BF07C0C901805F32
:1004C0009140809710F4419A3901EE244FE1439511
:1004D00001B212B290010426142612BA01BAF49E97
:1004E000F12CE49E1F0C70014A9500B232BB21BB77
:1004F00000940422E028469551F7112486010095C6
:1005000010950E211F210115110509F4C9CEC0E077
:10051000D0E0C5010C2E02C0880F991F0A94E2F7A3
:1005200080239123892B81F0C093F6009E01CE0198
:1005300063E0880F991F6A95E1F7220F331F820F3E
:10054000931F805A9F4FF5DD2196CF30D10509F7D3
:10055000A7CEAA1BBB1B51E107C0AA1FBB1FA61732
:10056000B70710F0A61BB70B881F991F5A95A9F75C
:1005700080959095BC01CD010895DC01CB01FC0173
:10058000E199FECF06C0FFBBEEBBE09A31960DB2FB
:100590000D9241505040B8F70895E199FECF9FBBAE
:0E05A0008EBBE09A99278DB30895F894FFCF93
:00000001FF
